:10000000052800000000000009005530B5213E30F1
:10001000B9219E003F30B9218C0010308D007E2127
:100020008D0B0F289F011F281630B921242117306E
:10003000B92124211F2890302421003024210530AB
:100040009F13102121080E3A031945281C3A031961
:100050005428323A0319EC28123A03197928063A3F
:100060000319AE28743A0319C62805309F17FF20DC
:100070007E21A1183F289921A40B3B2842287E21EC
:10008000A40B3F287E217E211F280C1C3528210827
:10009000242108308D0000308E000E08B921242163
:1000A0008E0A8D0B4D281B282208013A031D352886
:1000B00005309F17FF202408033E8E0010210C1DE1
:1000C0006D281030B921B3001130B921B4001230BD
:1000D000B921B5001330B921B6008C1D7528143034
:1000E000B921B7001530B921B8000E089F13FF20C1
:1000F0001F289F1E99288C1C35282208013A031DB1
:10010000352805309F17FF202408033E8E0010215C
:1001100008308D0008308F00223084000F08B9218C
:100120008000840A8F0A8D0B8E280E089F13FF20F3
:100130001F281F1E35288C1E35282208031D352830
:1001400005309F17FF202408033E8E001021023047
:10015000AA008930AB009B30AC00952805309F1772
:10016000FF207E212530840099218000840AA40B81
:10017000B4288E00250803199F16031D9F120E0731
:10018000053A03191F16031D1F1242280C1E35289D
:100190003830B92122058E003930B9210E060319F5
:1001A000E4283A30B92123058E003B30B9210E06F0
:1001B0000319E4283C30B92124058E003D30B921D3
:1001C0000E060319E4283528210824219F131F1740
:1001D000240810211F1314289E1B352821082421D0
:1001E00023088F009F1324088E00102120308400E4
:1001F0000008BF21840A8F0A8E0BF8281B288D0067
:100200002030840006298D002530840000089F1FBF
:100210000E295121840A8D0B0629080024210A2960
:100220008D002030840017298D00253084009F1F09
:100230001F296C211F1F21298D0B172908003F2121
:100240001A298000840A1C2996003230B5217F309B
:1002500066009701861308309400B421960C160CA2
:100260008039970606068606940B2D29B4211708B7
:1002700006068606B421FF3066004F30B529861B7E
:100280003F292A30B521093094000310861B03143E
:10029000960CB421940B4529960D2830B5211608EB
:1002A000080096003230B521FE3066009701061036
:1002B00008309400B42101301605960C9706060606
:1002C0008606940B5A29B421170806068606B4211F
:1002D000FF3066004F30B52906186C292A30B52149
:1002E00009309400031006180314960CB421940BE3
:1002F0007229960D2830B5211608080006187E29A7
:100300000E30B5217F3066008613B4210930940089
:10031000031006188D2986138F2986170314960C4F
:10032000B421940B8829FF306600B421960D16087D
:100330000800861B99290E30B521FE306600061094
:10034000B421093094000310861BA8290610AA299D
:1003500006140314960CB421940BA329FF306600F5
:10036000B421960D160808001A309500950BB62991
:1003700000348900831608148312080808008316C5
:100380008818C029831288000F08890083168B13F0
:10039000081555308900AA30890088148B17081178
:0403A00083120800BC
:1007F00050006C0069006E006500750073003100E8
:084000000000000001000A00AD
:02400E00F93F78
:1042000000001100000000002200330044005500AF
:104210000000050080000000000000003100DE000A
:104220005000500055004100460046009000FF003D
:10427000FF001100FF00B000FF00000000001F0061
:00000001FF
